:020000040800F2
:10500000F81B0020D5500008A9860008397E00084A
:105010000000000000000000000000000000000090
:10502000000000000000000000000000F5870008FC
:105030000000000000000000AB8600088588000822
:10504000E7500008E7500008E7500008E750000864
:10505000E7500008755C0008E7500008E7500008BA
:1050600000000000E7500008A15B0008E7500008BE
:10507000E75000081983000800000000E75000080E
:1050800000000000E75000080000000000000000E1
:10509000E750000800000000E7500008E750000853
:1050A000E7500008E7500008E75000086990000842
:1050B000E7500008E7500008000000000000000072
:1050C0000348854600F0B8FC00480047E9A0000806
:1050D000F81B00200448804704480047FEE7FEE72D
:1050E000FEE7FEE7FEE7FEE721890008C150000861
:1050F00030B50B46014600202022012409E00D4670
:10510000D5409D4205D31D469540491B25469540F7
:1051100040191546521E002DF1DC30BDF0B51FB40C
:105120000646002082B005464024019100901BE015
:10513000019922460F46304600F068FB049A059B11
:10514000801A994110D310461946224600F04EFBB2
:10515000361A8F410197224601200021009F00F05E
:1051600045FB38184D4100902046641E0028DFDCC6
:10517000019B00982946324607B0F0BD03460B4319
:105180009B0703D009E008C9121F08C0042AFAD2FD
:1051900003E00B780370401C491C521EF9D2704783
:1051A000D2B201E00270401C491EFBD270470022BF
:1051B000F6E710B513460A4604461946FFF7F0FF16
:1051C000204610BDF8B502464A40D40F42004B00BD
:1051D00052085B089A4202D20246084611464A002B
:1051E00023D0C30D4A00DDB2120EAD1A202D35DAE0
:1051F00049020126490AF6058A19002C00D05242BC
:1052000020214F1B1146B9402A411018C20D9A4265
:1052100021D0002C17D0012D08DCDA05801AD20F1E
:105220008019D207DBB200F01DFBF8BDDA05801A49
:10523000012340001B06C01880185A428018CA0F6C
:105240001043490007E04908C2071143DA05801AF4
:1052500080194008801800F0FDFAF8BD61000122B5
:10526000511A001BF7E70122D2075140AAE7012299
:10527000D2075040A6E770B502464A40D50F40001D
:105280004A00ED0740085208002814D0002A12D026
:10529000C40DD30D41020120C0055202490A520A31
:1052A000E41A091812187D34914201D3641C00E0FD
:1052B0004900002C01DA002070BD0023914201D387
:1052C000891A0343400849000028F7D100290AD071
:1052D000914202D10121C90705E0914201D2012189
:1052E00001E00121C943E005C018401900F0B2FAFD
:1052F00070BD420005D04200120E52428A4201DBCC
:1053000000207047C905081870470000F0B507462F
:105310000846584087B0C00F049048000E46590018
:1053200040084908BC1A884105D2384631461E4615
:1053300017460B4602465800400810434CD0300D2B
:10534000039040055900400D490D0590401A029008
:10535000402872DA18030121000B09050843019067
:1053600004980092002805D00199524200208841FB
:1053700000920190029840210A1A0199009800F0C9
:1053800035FA05460C466B4607CB00F050FAC019BB
:105390007141039A0E0D0023D71756401A467A40E2
:1053A000164344D0049A002A2DD0029A012A039A67
:1053B00015DC1205C01A914101263605001C714109
:1053C000D20F059ED2070093019202962A462346E9
:1053D00000F08EFA07B0F0BD38463146FAE7160500
:1053E000224A0F46B218C01AB74101210905001C14
:1053F0004F4100187F41114618187941E20F1043C0
:105400006D19644113E0E2076D0815436408C20793
:105410001443039A01261205C01A91413605001C57
:105420007141CE07400830434908C01851412A460F
:10543000234600F050FACDE7FFE704980122400030
:10544000C117121A00238B4104983146C417381A29
:10545000A141EEE730B40124E407634030BC55E7D6
:1054600030B40124E407614030BC4FE70000E0FFA6
:10547000F0B51FB488B00B990998002448400999E9
:10548000C00F490049080991C0070B9900904900D5
:1054900049080B9109990898A64608431CD00B9916
:1054A0000A98084318D0099801244000420D48008A
:1054B000410D099824050003000B204309900B9827
:1054C0000003000B20430B9050181C494018002289
:1054D00001901446104605E0002001460DB0F0BDD5
:1054E000032801DA034600E003239C46C11A0AAEF2
:1054F0000AE05F0008ADED5B4F00F75B7D430027DE
:10550000AA187C41491C5B1E6145F2DD410004ABD9
:105510005A522104120C0A43240C401C0828DFDBD9
:10552000019802900099704601910090059B049AA1
:105530000799069800F0DCF9D0E700000DFCFFFFAA
:10554000F0B50C465C4085B0E40FE40703944C00D2
:1055500000266408590094464908024602962243F0
:1055600021D062460A431ED06200570D4A000E0346
:105570002303550D012402462C492405781B1B0BDF
:10558000360B401823432643614600901C46501AB0
:10559000B44103D30098401C009002E09218009898
:1055A0005B41002803DA0020014605B0F0BD002071
:1055B000012109050746864611E064461D46141B75
:1055C000B54106D36546521BB341744607430C43AD
:1055D000A646CD0740084908284392185B41054676
:1055E0000D43EAD11046184313D060461946504087
:1055F0007140084306D06046101AB34106D201221A
:10560000002306E000220123DB0702E00122D2434F
:105610005310009874460105381C6141029C039D9B
:105620000019694100F057F9BFE70000FD030000D1
:1056300070B54B005B0803430BD04B005C0D00269C
:1056400033466542B341D417AD1AA34102DB0020B3
:10565000014670BD12053018514170BDC217C10F0F
:10566000504010B54018CA079623002100F0FAF800
:1056700010BD10B500229623114600F0F3F810BDBE
:105680000EB5C217C10F5040CA0740180021054B84
:105690000293019200910A460B4600F029F903B0EB
:1056A00000BD0000330400000EB505490291002141
:1056B00000910A460B46019100F01AF903B000BDB3
:1056C00033040000410040020122400AD205090EC5
:1056D00080187F2901DA00207047962903DC962282
:1056E000511AC84070479639884070474A000903EC
:1056F0000123090B1B051943094B10B5520D9A42A2
:1057000001DA002010BD064B34339A4203DC9A1AAA
:1057100000F07CF810BD03495118884010BD00000E
:10572000FF030000CDFBFFFFC20FD207400040087F
:105730000BD0C10D0723DB01C91840020905400A3F
:105740001143C208400711437047002001467047CB
:1057500010B5002904DB0124E40740428C412146B6
:10576000002B04DB1C460123DB075242A3418B4282
:1057700000D1824210BD000010B5002904DB0124D5
:10578000E40740428C412146002B04DB1C460123E8
:10579000DB075242A341994200D1904210BD000064
:1057A000CB0FDB07490010B5490802460A4307D072
:1057B0000A0D07240903E401090B121B002A01DC6E
:1057C000002010BDC900440F0C43C100E018D205F1
:1057D000801800F03FF810BD0122D207002800DB3E
:1057E000101A002900DB511A8142704710B5202A97
:1057F00004DB0146203A9140002010BD9140202357
:105800009C1A0346E3401943904010BD10B5202A6E
:1058100004DB0846203AD040002110BD0B46D3409F
:10582000D0402024A21A91400843194610BD10B55B
:10583000202A06DBCB170846203A1041C1170B433C
:1058400006E00B461341D0402024A21A91400843A1
:10585000194610BD002904DA401C490001D1400856
:105860004000704770B40024050C05D110240004DA
:1058700002D1002921D01124050E01D100020834E3
:10588000050F01D10001241D850F01D18000A41C4A
:10589000002801DB4000641C002908D020252E1BB5
:1058A0000D46F540A14000D00121294308430106DF
:1058B0001B1B000ADB1D02D5002070BC7047DB05F6
:1058C000181880180029F8DA401C4900F5D170BC7E
:1058D00040084000704710B5002B08DA0024401C37
:1058E000614192185B411A4301D14008400010BD4C
:1058F000F0B51FB482B005460C0003D0084603F093
:1059000067FC02E003F064FC203002460090214670
:105910002846FFF76BFF049B059A04460F46184381
:105920001143084314D0184610431BD0009840215F
:105930000A1A18460599FFF769FF05460E46009AB0
:1059400005990498FFF752FF084305D0012004E0B1
:105950002046394607B0F0BD0020C11705430E436D
:105960002C43374300990E986305401A7905E40AE1
:1059700000220C43FD0A0A3002D500200146E9E767
:105980000105101969410C9C0D9D00196941FFF733
:10599000A2FFDFE7FEB500231A461B1A8A4103DB8C
:1059A0000020014603B0F0BD4A000D0301212D0B7C
:1059B0000905520D0D43D10702D100186D41521E49
:1059C0005110FF31FF310131002704463E46384671
:1059D000009701910246012100200905FFF716FFFB
:1059E000C3197141F818324684468E464A416146D1
:1059F0002846611A904104D36046241A95417646A0
:105A00001F46241900986D41401C00903428E1DDA8
:105A1000F91930467041091BA84103D20022D24334
:105A2000134601E00022134601980105381C71411C
:105A3000FFF751FFB6E70000064C0125064E05E0D2
:105A4000E36807CC2B430C3C98471034B442F7D39F
:105A5000FFF73AFB28AF000848AF000870B58C1874
:105A60000578401C6B075B0F01D10378401C2A119D
:105A700006D10278401C03E006780E70401C491CD9
:105A80005B1EF9D12B0705D40023521E0DD40B70D9
:105A9000491CFAE70378401CCB1A921C03E01D78DE
:105AA0000D70491C5B1C521EF9D5A142D8D30020B1
:105AB00070BD000038B50446064805490068FFF788
:105AC00017FB604300E0401E00900028FBD138BD6A
:105AD00040420F0080010020F8B50446006881684C
:105AE0008907890F012902D10168C90722D181687C
:105AF000114A10261140012500290ED18168294341
:105B000081600120FFF7D6FF00F070FF07460CE030
:105B100000F06CFFC01B0A2807D9606D3043606538
:105B2000A06D2843A0650120F8BD20680068C0432F
:105B3000C007EDD10020F8BD170000801FB50B484D
:105B400000900B4801900B4802900B480390694667
:105B50000A4803F0B5FE0A4A08481146083903F01E
:105B60009DFD00F0B7F9002004B010BD31AD000874
:105B70000DAD00086DAD00086BAD00088C01002074
:105B80001000002010B500231A4603E0845CE318DF
:105B90009BB2521C8A42F9D3D84380B210BD000098
:105BA00010B5034800F0DEFC024800F0DBFC10BD3D
:105BB000941700204C17002030B5446C1C252C4055
:105BC0000125A540046C6560046863608368102B40
:105BD000036803D099600068C26030BD9A600068B5
:105BE000C16030BD1449012048720A4602205E326D
:105BF000507203203C3A507204200E3A50720F4803
:105C00000D4B0078087022310870203108770C495C
:105C10005A1C087858714978997123331871597151
:105C2000203318775977107551751A461E32107542
:105C30005175107651767047E41100203E01002026
:105C40006001002010B502F0ABFD202002F010FE34
:105C5000012004F089F8054803F06AFF044804F0C5
:105C60007FF9002004F086F910BD0000000100203B
:105C700083800000F8B502F009FE0520012100072D
:105C800000F0A0FE0025144C002800D06560134EE3
:105C90000221304600F096FE002815D10120207028
:105CA0000F48808F00280ED00127BF0200223946FE
:105CB000304600F094FE0A2003F061FC01223946D0
:105CC000304600F08CFE6560012000F0B3FD02203C
:105CD00000F0B0FDF8BD00006C0100200004005091
:105CE000E40D00207047000010B5084900224A6109
:105CF00007494B684C1523434B604B6808242343EA
:105D00004B60C009C001026010BD0000DC1700201C
:105D1000002002407FB500250C460646039500F0A2
:105D200059FDE009029003A901960095684600F02C
:105D3000E9FC002804D000F021FD002004B070BD73
:105D400000F01CFD0120F9E710B5002302E0C45C5F
:105D5000CC545B1C9342FAD310BD000010B5214A0D
:105D600000219069C305204804D5416902231943E5
:105D70004161911593699B0505D54369012423432E
:105D800043616302194393695B0505D543690824A0
:105D900023434361E301194393691B0505D5436917
:105DA0000424234343616302194393699B0405D58B
:105DB00043691024234343616302194393699B039E
:105DC00004D5446920231C43446119439369DB03D0
:105DD00005D54369402423434361A00201439161F7
:105DE00010BD000000200240DC17002070B5054601
:105DF00000F0FCFD0646184C0AE0681C08D0002D97
:105E000004D000F0F3FD801BA84201D9032070BD2F
:105E1000A069C007F1D1A069800701D50220A06167
:105E2000A069C00511D4A06980050ED4A069400501
:105E30000BD4A069000508D4A069800405D4A0692A
:105E4000800302D4A069C00303D5FFF787FF0120B8
:105E500070BD002070BD000000200240F8B517465C
:105E6000002605460C4600F0B5FC09E02946022054
:105E7000226800F091FC002804D1241D2D1D361D40
:105E8000BE42F3D300F07AFCBE4201D20020F8BD3E
:105E90000120F8BD10B500F09AFD10BD10B50948FD
:105EA00000F0BAFF80B2FFF7FFFB074A074BFFF78E
:105EB000DFFA0022064BFFF743FBFFF717FC80B227
:105EC00010BD000000160020F853E3A59B843E405F
:105ED00000408F4010B5144C144822461032114631
:105EE000083903F0DBFB0022114BE168A068FFF7E3
:105EF00027FB104A104B04F0ABF900220F4BFFF7C1
:105F0000AFFA00220E4BFFF7B3FAFFF749FC20600F
:105F100000221346E168A068FFF71AFC01D0206850
:105F200010BD0020206010BD000000208C0100206A
:105F300000AA8F406C45D9CC955BC83F0000F03F6C
:105F400040A5E54010B5084800F096FA0A21064839
:105F500000F032FA044800F01DF9800503D502482C
:105F600000F01AF980B210BDA4150020F8B52F4D2D
:105F700000220121284600F032FDFFF7E3FFFFF782
:105F800078FB2B4E3146FFF776F92A4C0122A060B0
:105F90001146284600F023FD2749A06800258842C5
:105FA0003EDB2078254F002815D02570FFF7CAFF6B
:105FB000FFF75FFB3146FFF75EF9A060FFF7B4FB28
:105FC00000223B46FFF746FA00221D4BFFF750FA2E
:105FD000FFF7E6FB6060A068FFF7A6FB00223B46E8
:105FE000FFF738FA174A184BFFF742FA06460F46F2
:105FF0006068FFF799FB134A144B5242FFF738FAD7
:1060000032463B46FFF782F9FFF7CAFB1049606052
:10601000884201DD616004E0FF21C905C84200D368
:1060200065606068FFF74EFBC0B2F8BD0004005029
:1060300000401B44480000200000604000000C406D
:1060400000E064403333333333B33040CCCCEC3FE7
:106050000000C842F8B5054604464035287C0026B5
:10606000012808D001202874206881688907890FD9
:1060700001290ED101E00220F8BD0168C90708D04E
:10608000606D202108436065012600202874304699
:10609000F8BD616DFF220132914302221143616517
:1060A000C1688907890F0091C16889088900C160AA
:1060B0002068816892071143816000F097FC0746D1
:1060C0000EE000F093FCC01B0A2809D9606D022184
:1060D0008843102108436065002028740120F8BD22
:1060E000206880680028ECDB2068C168009A1143B2
:1060F000C160606D80088000401C6065C5E70000DD
:10610000F8B506460D464036317C01290DD00121F7
:10611000317401688A68520709D5416D2022114304
:106120004165002030740120F8BD0220F8BD174BF6
:106130006A68D80547109A42154C8A6A2B6812D0B3
:106140005B035B0B1A438A622968490305D5A16882
:106150000143A1600A20FFF7ADFC2868800312D537
:10616000A06838430EE05B035B0B9A438A622968A0
:10617000490302D5A1688143A1602868800302D544
:10618000A068B843A06000203074F8BD0110000082
:1061900000270140406D70470068006C70470000A8
:1061A00070B5040006D0606D2646002540360028F4
:1061B00002D006E0012070BDA5653574204600F0D0
:1061C000D3F8606DC00603D421688868400705D500
:1061D000606D1021084360653574EBE7606DFF2248
:1061E0000132904302221043606588688207920F53
:1061F0005B48012A02D10A68D2072BD103236268C7
:106200009B079A4205D05B429A4202D05B009A42B9
:1062100009D10A69920092080A6121680A696368D3
:106220001A430A610CE00A69920092080A618168C7
:106230000F229204914381608168626811438160FA
:106240002168CA6818239A43CA602168CA68A3688B
:106250001A43CA60816801225206914381608168B5
:10626000A28E52061143816020688168C90004D45F
:10627000816801221207114381602068C168394A90
:106280001140C1602069E168022825D00020014347
:10629000204620300278037B52035B001A431143EF
:1062A000226B1143A26992031143E269D2031143A5
:1062B0002268D3681943D160616A0A46FF3AC23A3C
:1062C00005D0A26A11432268D3681943D16042788D
:1062D0000121012A02D00BE00420D8E70078002831
:1062E00023D0606D202210436065A06D0843A06537
:1062F000E06B012820681FD00169C90703D001693C
:1063000049084900016120684169C908C900416123
:1063100020684169A26B11434161A565606D8008E9
:106320008000401C6065002070BD2068C2680123A9
:106330001B041A43C260DBE70269FF239B009A43F8
:10634000026120680269236CA66C1A43636C3343B4
:106350001A430261206802690A430261D3E7000020
:10636000002701401902FEFF10B586B00446142133
:106370006846FEF71CFF0E492068884216D10D487A
:10638000416B421511434163C16A01221143C1624D
:10639000C06A6946104005900220009003200190D9
:1063A000002002900520000700F050FA06B010BD52
:1063B0000024014000100240F8B50446406925461B
:1063C00040350E4608280BD02068C068C00709D0A9
:1063D000606D202108436065002028740120F8BD0D
:1063E000082700E00C2700F001FB009011E0701C72
:1063F0000FD0002E05D000F0F9FA0099401AB042F3
:1064000007D9606D042108436065002028740320CB
:10641000F8BD206800683842E9D0606D012149026A
:10642000084360652068C16809058A0F0C21002AAD
:106430001BD12022125D002A17D10268120714D541
:10644000826853070122002B08DB43688B434360BB
:10645000606D130298431043606506E0606D202371
:1064600018436065A06D1043A065A069002801D1A4
:10647000206801600020F8BD70B504462168002046
:106480008968490721D425464035297C01291CD03B
:1064900001212974E169012904D02046FFF71CFB82
:1064A000002811D1616D0A4A1140FF2201321143C7
:1064B00061650021A165297422681C211160216891
:1064C0008A6804231A438A6070BD022070BD0000F0
:1064D000FEF1FFFF30B5014620314A790023022A40
:1064E00004D00422C2630B71012030BD026814681D
:1064F0000E25AC43146002681468640864001460DC
:10650000446C1C22144001221546006CA5404560D5
:106510004A7118460B7130BD70B500240146203118
:106520004A79022A03D00421C163012418E00268D9
:1065300013680E25AB431360026813685B085B00A9
:106540001360436C1C221340012215469D40036CCE
:106550005D604A7100220A71816B002900D0884772
:10656000204670BDF0B4016C0D6801680C68466C83
:106570001C2304221E401746B7402F420ED0670747
:106580000CD50C68A40602D40C6894430C60416CD2
:1065900019408A40016C4A60016B1AE00227B7403B
:1065A00002462F402032002F17D0A70715D50C68C0
:1065B000A40605D40C680A25AC430C600121517176
:1065C000446C02211C40036CA140596000211171F0
:1065D000C16A002918D0F0BC08470827B7402F42ED
:1065E00012D0240710D50C680E25AC430C60446C07
:1065F00001211C400B46A340046C6360C1635171D0
:1066000000211171416BE4E7F0BC704770B50400E4
:106610003CD01F48256814212818FEF769FD80002A
:1066200060641C48206402212046203002464171EB
:1066300029681948E3680140A0686669184323691E
:1066400033431843A3691843E3691843236A184383
:10665000084328600121A0688903884210D00D48B2
:106660008030836A656C1C210D400F26AE40B34319
:106670008362656C63680D40816AAB400B43836243
:106680000020E06301215171107170BD012070BDC7
:10669000F8FFFDBF000002400F80FFFFF8B5044681
:1066A0008C46203001790025012909D00126067188
:1066B00041790027012905D0077102252846F8BD38
:1066C0000220F8BD02214171E76320680168490892
:1066D0004900016061462046FFF76EFA206B0028F2
:1066E0002068016801D00E2205E004229143016078
:1066F000206801680A221143016020680168314363
:106700000160DBE7F8B51A4E0546307C0F460128DC
:1067100007D0012030741748FFF768FB010002D052
:1067200021E00220F8BD0020C04338606C6814E00E
:106730002046FFF7D9FA0F48FFF758FB01460E48ED
:10674000426808239A434260426843159A43426074
:10675000002901D03C6006E08034A8686A68C00166
:106760008018A042E4D8002030740846F8BD00002C
:10677000DC17002050C3000000200240054841689B
:10678000022211434160416801221143416000200F
:106790007047000000200240F8B50C4C1646207CE3
:1067A0000F46012808D0012020740948FFF71EFB7E
:1067B0000025002802D006E00220F8BD65613E6099
:1067C0000348FFF713FB2574F8BD0000DC17002019
:1067D00050C3000011484168C9070BD0EFF3108186
:1067E00072B60F4AC2600F4AC26081F310884168D6
:1067F000C9070ED1416889070DD5EFF3108172B634
:10680000094A0261094A026181F3108840688007E1
:1068100001D5012070470020704700000020024091
:10682000EFCDAB8905040302BFAE9D8C1615141382
:106830007047000010B504494A69024202D048611D
:10684000FFF7F6FF10BD000000040140FCB5002377
:106850000124A2E027462A469F403A406FD04D6867
:10686000012D05D0022D03D0112D01D0122D16D1EE
:1068700085680326AC465D00AE46AE406546B5432E
:10688000AC46CE687546AE4065462E438660466887
:106890000D79BE43ED06ED0F9D4035434560C6685A
:1068A0005F000325BD40AE46AE4335468E68BE4010
:1068B0002E43C6604E68022E01D0122E14D1DE087F
:1068C000B60036180196366A5D07B446EE0E0F25FF
:1068D000B54000966646AE43B4460D69009EB5408D
:1068E00066462E43019D2E6206687546AE430D79BD
:1068F000AD07AD0FBD40354305604D68ED004BD58C
:10690000294D6E6B26436E639E08284DB60075199F
:10691000AC46AD689E07360F0F27B740BD4305272D
:106920003F07B84201D1002715E0214FB84201D1FD
:10693000012710E01F4FB84202D102270BE02BE0E5
:106940001D4FB84201D1032705E01C4FB84201D1C9
:10695000052700E00627B7402F436546AF60184D76
:106960002E684F689643FF0300D516432E606E686D
:106970004F689643BF0300D516436E60AE684F68FC
:106980009643FF0200D51643AE60EE684F6896430B
:10699000BF0200D51643EE605B1C0A681546DA405C
:1069A00000D057E7FCBD000000100240000001408D
:1069B0000004005000080050000C0050001C005063
:1069C000000401400069084000D00120704742697E
:1069D00013460B401B0491430B4383617047002A0D
:1069E00001D0816170478162704700000148806872
:1069F00070470000740100200248816802788918FD
:106A0000816070477401002010B5084800240168B7
:106A1000402211430160204600F00AF8002801D00E
:106A2000012401E000F042FA204610BD002002409F
:106A300070B504460D4D7D202978C000FEF758FB47
:106A400001460B480068FEF753FB00F02BFF0028BF
:106A500009D1042C07D200222146401E00F04EFA34
:106A600000206C6070BD012070BD0000740100202A
:106A70008001002070477047F8B501F007FF604CB7
:106A80000120E070208AFEF7F4FD01467F20C0055A
:106A9000FEF7F1FB5B4D06462968FEF793FB286085
:106AA0000120A16AC005814201DA084603E03046B0
:106AB000FEF7DDFBA062FF21C9050025C84200D317
:106AC000A562607800280BD102214F48FFF77AFFBA
:106AD00002004E494E4817D00022FFF780FFE562C2
:106AE00002214948FFF76EFF4A4E002855D0E56263
:106AF000B08AFEF7BEFD434F3968FEF76DFE5FD2E8
:106B00004549012008705DE00122D1034048FFF7AC
:106B100066FF208AFEF7ADFD01467F20C005FEF727
:106B2000AAFBE16AFEF74EFB3C49E0628842D7DDF2
:106B300038480127F926403000900A213046FEF7F8
:106B4000D7FA002903D131493148FFF7A3F90221CF
:106B50002D48FFF737FF002801D0002701E0002F64
:106B600012D102212848FFF72DFF00280CD103F095
:106B700037FB00990120888004F08EF8642002F031
:106B8000FEFC28492648C8600A2002F0F8FC30467E
:106B9000761EF6B20028D0D1A2E7208AFEF769FD62
:106BA00001467F20C005FEF766FBE16AFEF70AFB9F
:106BB0001D49E06288429BDB1A491948C86097E783
:106BC00015480570708F401EFEF748FD3968FEF7C6
:106BD00003FE06D82079002803D01449012008704C
:106BE00001E012480570708FFEF743FD3968FEF72B
:106BF000F3FD04D22079002801D003F0B5FAF8BDE6
:106C00003C010020700100200004005000800000C2
:106C100000000050E40D00207600002000004040FD
:106C20000400FA0500ED00E00000A040860000200E
:106C3000704770B5040010D0022025462035A87397
:106C4000204601F071FBA87B032805D0204600F008
:106C5000B9F80020A873687370BD012070BD70473B
:106C6000704710B5044600680168C943C90708D1D8
:106C70008168C943C90704D1012141602046FFF75B
:106C8000FBFE20680168C943890708D48168C943AD
:106C9000890704D4022141602046FFF7EBFE2068FB
:106CA0000168C943490708D48168C943490704D426
:106CB00004214160204600F0F7F820680168C943CC
:106CC000090708D48168C943090704D40821416031
:106CD0002046FFF7ADFF20680168C943C90608D404
:106CE0008168C943C90604D4102141602046FFF7DA
:106CF000C2FE20680168C943890608D48168C94377
:106D0000890604D4202141602046FFF7A9FF2068AE
:106D10000168C943490608D48168C943490604D4B7
:106D2000402141602046FFF79AFF10BDF8B50400EE
:106D300005D025462035A87B002802D006E001209A
:106D4000F8BD00206873204600F04EF80220A873BA
:106D50002068C26884466368012B01D10620824303
:106D600016486169814202D0072040038243002B0C
:106D700001D1D82082431248A66802401846304309
:106D8000676A266A3E433043A66A30431043002BAD
:106D900002D0012B04D005E02369E2691A4300E028
:106DA000E2681043054A914202D0A26911430843A8
:106DB0006146C8600120A8730020F8BDFFFF0000F5
:106DC000F8F119FF10B500680549884207D1054858
:106DD000816B4900490881630D2000F073F810BDF4
:106DE000007C00400010024010B50068084988424D
:106DF0000CD10848816BC204114381630022012138
:106E00000D2000F07BF80D2000F06CF810BD0000A4
:106E1000007C0040001002400068C069704700001C
:106E2000F8B504460220254620351746A8731D48AC
:106E30000268C3041A4302602068C2689B121A43A6
:106E4000C260206802690126324302612268102074
:106E50005060206881611021204601F0D5FA032896
:106E60001FD021680820486020684761082120461B
:106E700001F0CAFA032814D0204601F055FAA87B85
:106E800003280ED020688168314381602068016941
:106E90003143016120680169042211430161AE732D
:106EA0000020F8BD00040140704700000448416B19
:106EB000012211434163816B0204114381637047D6
:106EC00000100240002809DBC106C90E01208840DD
:106ED00003490860BFF34F8FBFF36F8F7047000007
:106EE00080E100E0002805DBC106C90E01208840D2
:106EF000014908607047000000E100E010B502F0B1
:106F0000B9F910BD02494A6882434A6070470000DF
:106F1000007000400248016882151143016070470B
:106F20000070004002494A6802434A60704700000E
:106F300000700040054801680222114301600448C6
:106F4000016904221143016130BF704700700040A5
:106F500000ED00E0F0B5154A1368154D54152D6A83
:106F60002340ED07ED0F002B04D0002D02D0166852
:106F7000A64316601668B608B600064316600D48AC
:106F8000076904263743076101290DD040BF20BFA0
:106F900020BF0169B1430161002B04D0002D02D054
:106FA000106820431060F0BD30BFF2E70070004071
:106FB0000000014000ED00E0F8B50446007800272D
:106FC000534D800671D5524E403EB06BC00004D484
:106FD000B06BA9050843B06301274E480168C90595
:106FE00011D40168821511430160FFF7FFFC009086
:106FF00005E0FFF7FBFC0099401A642837D84548A4
:107000000068C005F5D532680321090560680A40AB
:107010000140914208D08103890F032904D13168CE
:10702000890301D50120F8BD2A69032109040A401A
:1070300022D0084090421FD0207880061CD52869B5
:107040002A6988430121C9040A432A612A698A43BB
:107050002A612861C0050FD5FFF7C8FC009008E041
:10706000FFF7C4FC0099411A2B48814201D9032043
:10707000F8BD28698005F3D561688803800F03286F
:1070800005D132680005824301400A433260286915
:10709000032261681204114008432861002F04D0C4
:1070A000B16B012000078143B1632078C00705D090
:1070B000E868A168800880000843E86020788007BD
:1070C00005D5E8680C218843E1680843E86020782A
:1070D000400706D5E86803218902884321690843EF
:1070E000E8602078000706D5E86803210903884393
:1070F00061690843E8602078000606D5E868032146
:1071000089048843A1690843E8600020F8BD0000B5
:10711000401002400070004088130000F8B50E4691
:10712000050038D05E480068C007C00FB04214D2D6
:107130005B4C20684008400030432060FFF756FC5D
:10714000074605E0FFF752FCC11B564881427AD83A
:107150002068C007C00FB042F4D12878524C800795
:1071600005D5E068F0218843A9680843E0602878E5
:10717000C00752D06868022806D0032807D02168CB
:1071800001280AD0890504E02168890301E021680B
:107190008901002903DB0120F8BD4907F9E7E1680F
:1071A000890889000143E160FFF720FC0746686811
:1071B00002280AD0032814D001281ED029E0FFF7A6
:1071C00015FCC11B374881423DD8E0680007800F9D
:1071D0000228F4D121E0FFF709FCC11B31488142AC
:1071E00031D8E0680007800F0328F4D115E0FFF7DD
:1071F000FDFBC11B2B48814225D8E0680007800FAA
:107200000128F4D109E0FFF7F1FBC11B25488142B9
:1072100019D8E0680007800FF5D121480168C90737
:10722000C90FB14217D901684908490031430160CB
:10723000FFF7DCFB074608E005E0FFF7D7FBC11BC3
:107240001848814201D90320F8BD15480068C007DD
:10725000C00FB042F1D12878400706D5E068072179
:1072600009028843E9680843E0602878000707D5E9
:10727000E0680721C90288432969C9000843E06022
:1072800000F03AF8E168094A0906090F515CC84064
:107290000749086007480068FFF7CAFBF8BD00000F
:1072A00000200240881300000010024072AE000867
:1072B0008001002078010020044805490068C96861
:1072C000044A4905490F515CC840704780010020BD
:1072D000001002408BAE0008044805490068C968E8
:1072E000044A8904490F515CC8407047800100205E
:1072F000001002408BAE000870B51A4AD3681A49D4
:107300000C2018408D0004280CD04E00082810D006
:107310000C2810D050680004410F0120C003491C04
:10732000884070BD1068C00601D5084670BD28466B
:1073300070BD304670BD98020C4C000F205C1B02E3
:107340009C0FD368641CDB0301D5314603E012684F
:10735000D20600D4294601F052FF22460023FDF751
:10736000DDFE70BD0010024000093D0082AE000845
:10737000FEB505007ED0FE4CE7680C20E6680740AD
:107380000120000406402878C00747D0082F05D008
:107390000C2F0AD101200004864206D12068800308
:1073A0003CD568680028E5D038E001206968000411
:1073B000814203D121680143216011E005230122AC
:1073C0001B0492049942216802D111432160F1E724
:1073D0008143216021680140009120689043206032
:1073E000686800280DD0FFF701FB009005E0FFF76B
:1073F000FDFA0099401A64287BD820688003F6D5EE
:107400000CE0FFF7F3FA009005E0FFF7EFFA0099C0
:10741000401A6428F0D820688003F6D428788007C2
:1074200056D50923E868042F0DD00C2F01D1002E6A
:1074300009D000283CD02168994301432160FFF71F
:10744000D5FA064628E02168490701D5002891D0E1
:1074500061681F22120291432A691202114361607E
:107460002168994301432160FFF746FFE16809065F
:107470000A0F00E08BE1BF49895CC840BE49086043
:10748000BE480068FFF7D4FA002873D120E0FFF768
:10749000ADFA801B0228AFD820684007F7D5606896
:1074A0001F210902884329690902084360600FE02F
:1074B0002068400840002060FFF798FA064604E084
:1074C000FFF794FA801B022896D820684007F7D46B
:1074D0002878C00660D5002F0CD0A86900284AD0B3
:1074E0002068FF21013108432060FFF77FFA06463C
:1074F0002EE0C1E02068800502D5A8690028A6D04A
:107500006068072149038843296A0843606060680E
:10751000297F0002000A090608436060286A410BBF
:107520000120C003491C8840E16809060A0F9149FF
:10753000895CC8409049086090480068FFF778FA75
:10754000002817D128E0FFF751FA801B0228A2D8A3
:1075500020688005F7D56068072149038843296AB8
:10756000084360606068297F0002000A090608433A
:10757000606011E0E2E02168FF200130814321607A
:10758000FFF734FA064604E0FFF730FA801B0228C2
:1075900072D820688005F7D42878794E000724D562
:1075A00068690028306910D0012108433061FFF775
:1075B0001DFA009005E0FFF719FA0099401A022819
:1075C0005AD830698007F6D50FE040084000306196
:1075D000FFF70CFA009005E0FFF708FA0099401A4F
:1075E000022849D830698007F6D42878400766D544
:1075F00000200290A06BC00006D4A06B01210907F7
:107600000843A063012002905E480168C90511D4B7
:107610000168821511430160FFF7E8F9009005E069
:10762000FFF7E4F90099401A642825D85548006806
:10763000C005F5D5FF20AA680130824203D1316927
:107640000143316111E001218902002A07D005239D
:107650001B029A4203D132690A433261EFE7326971
:1076600082433261306988433061A868002810D0B5
:10767000FFF7BCF9009008E05FE0FFF7B7F90146BB
:107680000098091A4048814257D830698005F4D5DE
:107690000DE0FFF7ABF9009006E0FFF7A7F90099BE
:1076A000411A3948814248D830698005F5D402989A
:1076B000002804D0A06B012109078843A063686AF1
:1076C000002866D00C2F3ED00126360602282068FE
:1076D00005D0B0432060FFF789F905462FE0B0439D
:1076E0002060FFF783F9074604E0FFF77FF9C01B2E
:1076F000022822D820688001F7D4E96AA86AE268E3
:107700000843296BFD231B049A4311430843E0609F
:10771000206830432060FFF769F9054604E0FFF771
:1077200065F9401B022808D820688001F7D530E0B1
:10773000FFF75CF9401B022801D90320FEBD206839
:107740008001F5D425E00128F8D0E0680121090482
:10775000AA6A014091421AD10F218904EA6A0140C4
:10776000914214D1032189050840296B88420DE01C
:107770000010024072AE0008800100207801002055
:1077800040100240007000408813000001D001202A
:10779000FEBD0020FEBDF8B504000ED0FF27606AD4
:1077A0000537002500280AD0256165612646403648
:1077B000A562707C002807D00AE00120F8BD60684F
:1077C000B842F3D0E561F1E73574204600F03EF8A9
:1077D000022171742068026840239A4302602123C9
:1077E000A26860689B021A4038401043E3688A022E
:1077F0001340184323690B40217D1843C907C90F63
:107800000843A169931019400843E16938231940DE
:107810000843216A802319400843A16A9300194054
:10782000084321680860A0690421000C0840616ACF
:10783000102319400843216848602068C1699143BA
:10784000C1616565012070740020F8BD10B586B077
:10785000044614216846FDF7AAFC104920688842B6
:1078600019D10F48416B821411434163C16A01224F
:107870001143C162C06A002110400590E0200090D1
:107880000220019003200390029104910520694693
:107890000007FEF7DBFF06B010BD0000003001401E
:1078A00000100240094910B5401E884201D901204C
:1078B00010BD074C60610321081F01F0DBFC0020B4
:1078C000A06107202061002010BD0000FFFFFF0025
:1078D00000E000E070B505462C4602202034002967
:1078E00008D004290BD008290ED0627F012A10D0BD
:1078F000012070BDA27E012AFAD1A0760AE0E27EC4
:10790000012AF5D1E07605E0227F012AF0D1207727
:1079100000E060770122286801F02EF80122286833
:1079200092070121904205D0074A904202D0074AAF
:10793000904204D182685207520F062A02D0026890
:107940000A430260002070BD00080140001401409D
:1079500070B504460D460068002201F00DF820685D
:10796000016A0C4A114203D10168490849000160CB
:1079700001202034002D06D0042D06D0082D06D07D
:107980006077002070BDA076FBE7E076F9E720770E
:10799000F7E70000111100007047704770470000C2
:1079A000F8B502680446D06911689668814B0546AF
:1079B0001D402023002D6CD0F7077F4DFF0FBC46E4
:1079C0000D402F4379D02546C7078035002F06D0BC
:1079D000CF0504D5012717622A683A432A60820737
:1079E00008D5F20706D0276802223A622A680427DF
:1079F0003A432A60420708D5F20706D026680422D7
:107A000032622A68022632432A6002070AD50A46F1
:107A10001A406646324305D02668082232622E6834
:107A200016432E60020508D54A0106D501222668B4
:107A3000D20232622A681A432A602A68002A30D0A9
:107A4000800606D5880604D5616E002901D020463F
:107A50008847286821688968490602D42821084295
:107A600025D0204601F017F920688168490619D50C
:107A7000826840218A438260206F002812D04F49DB
:107A80008163206FFEF748FD00280AD0206F816BCC
:107A900006E0850611D58D060FD5616E77E020468C
:107AA0008847F8BD2046FFF779FFF8BD05E020467E
:107AB000FFF774FF00202860F7E7256E012D56D1EF
:107AC000C50654D5CD0652D51026166220688168A9
:107AD00025464906403500292ADA226F116849688F
:107AE0000904090CE1D02F8B8F42DED9698311681C
:107AF0000968890617D40168320191430160206842
:107B0000816849084900816020688168402291436A
:107B10008160E3670020206620680168B14301604E
:107B2000206FFEF7D7FC288B698B401A81B21AE0D0
:107B3000298B6A8B891A6A8B89B2002AB5D00029F1
:107B4000B3D00268FF252135AA430260206882680D
:107B5000520852008260E367002020666066206859
:107B60000268B24302602046FFF716FF9DE7C50298
:107B700008D5750206D50120000510622046FFF7E2
:107B80000CFF92E7050605D50D0603D5A16E002969
:107B900085D18AE7400688D5480686D511682046F3
:107BA0004024A143116083670021816600F043F9FE
:107BB0007BE700000F08000020010004BD8B0008D7
:107BC00010B5040003D0A06F002802D007E0012008
:107BD00010BD002174200155204600F027F8242014
:107BE000A06720680168490849000160204601F04B
:107BF000A5F80128ECD0606A002802D0204600F0E9
:107C0000C8FE206841680922D20291434160206881
:107C100081682A2291438160206801680122114312
:107C20000160204600F01AFF10BD0000F0B587B0DB
:107C3000064614216846FDF7BAFA2C493068884296
:107C400051D12B48416B0122920311434163C16A18
:107C500001221143C162C06A002510400590032033
:107C6000400200900220032701A9A1C10420049032
:107C7000052069460007FEF7E9FD1F4C1D48A56079
:107C8000E56081C48027E560A760202025616061F0
:107C90000002A0611848083CFEF7B8FC002801D09B
:107CA000FEF720F83467A662144C124821461438B7
:107CB00020600320606010200831A1C16561A561CA
:107CC000E56120462562FEF7A1FC002801D0FEF701
:107CD00009F8F466002201211B20A662FFF70EF9C5
:107CE0001B20FFF7FFF807B0F0BD0000003801408F
:107CF00000100240300002404C1700209417002072
:107D000070B5C36F202B27D100290BD0002A09D0D2
:107D1000012483682403A34206D10369002B03D105
:107D2000CB0701D0012070BD034660331C7D012CC0
:107D300012D001241C7500230366084C0368A3427B
:107D400007D05C68240204D51C680125AD062C43CD
:107D50001C6001F0F3F870BD022070BD00480040C7
:107D600070477047FFB50446806F83B017460D46D5
:107D700020285ED1002D0AD0002F08D0A168C001B4
:107D8000814207D12069002804D1E80702D00120F0
:107D900007B0F0BD204660300090007D012848D03B
:107DA0000098012101750020802108512120A06741
:107DB000FEF71CFE2646403601903782778201206E
:107DC000A1680003814202D12069002805D02F4616
:107DD000002500990020087511E00027F9E700222E
:107DE0008021204601F0F0F8002815D1002F15D091
:107DF0002168387888627F1C708A401E7082708A81
:107E0000019B002806980090E9D1002240212046DD
:107E100001F0DAF8002808D00320B9E728882168A3
:107E2000C005C00D8862AD1CE6E72020A0670020D9
:107E3000AEE70220ACE77047034D044C04A001F00C
:107E4000BDF9E560FAE700000400FA0500ED00E086
:107E5000486172644661756C745F48616E646C65FC
:107E6000722E0D0A0000000010B505242407002220
:107E700004212046FEF7B3FD002208212046FEF72C
:107E8000AEFD0A2001F082FB012204212046FEF70C
:107E9000A6FD0A2001F07AFB002204212046FEF70D
:107EA0009EFD10BD10B505242407002204212046A4
:107EB000FEF795FD012208212046FEF790FD0A20DD
:107EC00001F064FB012204212046FEF788FD0A2010
:107ED00001F05CFB002204212046FEF780FD10BD6E
:107EE000F8B500240526074625463607002204215A
:107EF0003046FEF774FD0A2001F048FB0122042100
:107F00003046FEF76CFD6006040E08213046FEF791
:107F100059FD002801D0641CE4B2052001F036FBB5
:107F20006D1CEDB2082DE1D3002F03D0FFF79CFFAD
:107F30002046F8BDFFF7B6FFFAE770B505260546FF
:107F40003607002204213046FEF749FD0024E809E7
:107F500001D0012200E0002208213046FEF73FFD5B
:107F60006806050E0A2001F011FB012204213046AB
:107F7000FEF735FD0A2001F009FB002204213046FE
:107F8000FEF72DFD0A2001F001FB641CE4B2082C71
:107F9000DDD370BD10B50524240701220821204639
:107FA000FEF71DFD012204212046FEF718FD0022E8
:107FB00008212046FEF713FD0A2001F0E7FA00220F
:107FC00004212046FEF70BFD10BD10B50524240743
:107FD000002204212046FEF702FD0022082120464F
:107FE000FEF7FDFC0A2001F0D1FA0122042120460F
:107FF000FEF7F5FC012208212046FEF7F0FC0A20DE
:1080000001F0C4FA10BD70B505252D07002401222A
:1080100008212846FEF7E3FC062001F0B7FA01220A
:1080200004212846FEF7DBFC062001F0AFFA07E04A
:10803000641CE4B2FA2C03D9FFF7C7FF012070BD1E
:1080400008212846FEF7BEFC0028F1D100220421B9
:108050002846FEF7C4FC002070BD0000F8B500F013
:108060002FFD00F05FFD5B480068C069FDF716FF5B
:10807000594C5A49A082898F594E0025002931D088
:10808000A26A730357499A4202DB02220A7000E097
:108090000D700A7801218902002A05D0012A0ED02C
:1080A000022A10D0032A1DD1608B01282ED002286D
:1080B00018D1484808214038FFF74AFC12E0FF2257
:1080C000F5329042F0D2608B01281DD0022804D0F6
:1080D00008E03046FEF783FC04E03E4808214038C3
:1080E000FFF7F8FBFDF742FF20700121C90230467F
:1080F000FEF768FC0127FF0300282DD03A480560F1
:10810000A079002804D007E00022E2E70122E0E79E
:108110000120A07100F0BAFF80213046FEF752FC2A
:10812000002806D0002208213046FEF758FC012224
:1081300005E0012208213046FEF751FC002205200F
:1081400039460007FEF74BFC244C284E4034A08CE7
:10815000274F012803D01CE0A5710022EAE725483B
:108160006946088072B680212348FDF7D3FD0028B8
:1081700004D0022269462048FDF770FE62B61FA0B7
:1081800001F01CF8A58402F087FD642001F0F7F9E6
:10819000FE60608C012808D110486584058002F0DB
:1081A0007BFD642001F0EBF9FE60208C012806D1F4
:1081B000258402F071FD642001F0E1F9FE600748BA
:1081C000124A0188914202D1C088002800D1FE6085
:1081D000F8BD0000C81600203C010020E40D00207E
:1081E0000004005084000020700100200400FA0503
:1081F00000ED00E0AAAA0000384A0008BDF8C8EB6C
:10820000C9FDBCB6C4A3CABD0D0A0000AA55000032
:1082100038B55721202000F07AF80321212000F002
:1082200076F84021222000F072F80821232000F087
:108230006EF8AA21302000F06AF81048018F142946
:1082400001D8002901D1012101870C4C40346188FB
:10825000142901D8002901D102216180008FC1B207
:10826000322000F054F8A178332000F050F868462E
:1082700000F006F80A2001F089F938BDE40D00206D
:1082800010B501460F2000F021F8002800D0012091
:1082900010BD10B50446FFF77DFE3220FFF74DFEFE
:1082A000FFF7B1FEE0B2FFF748FEFFF7ACFEFFF7C5
:1082B00071FE3320FFF741FEFFF7A5FE0020FFF718
:1082C0000FFE0446FFF781FE204610BD10B50C4698
:1082D000FFF7DFFF2070012010BD70B50D4604468A
:1082E000FFF758FE3220FFF728FEFFF78CFEE0B2C2
:1082F000FFF723FEFFF787FE2846FFF71EFEFFF776
:1083000082FEFFF762FE0A2001F040F970BD10B551
:10831000FFF7E3FF012010BD10B50248FEF7A1FCF6
:1083200010BD000000160020FEB50446002772B6FE
:10833000334A01688B1804D13248C768032080048F
:10834000074088680190C868009048698E69002BD2
:1083500008D12C4940398B6ACD042B438B628B6A40
:10836000AB438B62014631433CD025492368CB4265
:1083700005D12449CA6803239B049A43CA60254651
:108380002035002810D021680A6901231A430A61A8
:10839000216848610821204600F036F8032800D102
:1083A000A873216808204860002E10D02068016959
:1083B000012211430161206886611021204600F0EE
:1083C00023F8032800D1A8732168102048600C48C6
:1083D0002168C14206D10B48C1680322920491432F
:1083E0003943C16020680169490849000161216879
:1083F0000198886021680098C86062B6FEBD0000E0
:108400000084FFBF4010024070B506460B480D4681
:10841000002409490068FCF76BFE7D21C900484330
:108420003168401E00D103240B682A469A4301D0CC
:108430000028F6D1204670BD204E000080010020AB
:108440001CB5002116480091144A01910260C163D5
:1084500012054260816007228263012202610246A6
:10846000C16020321170FF235170C23343628162B8
:10847000117301638161042241634261C161FDF7AF
:108480008FFE084800908013019069460448FDF76C
:1084900037FE00210248FDF7DDFD1CBD0024014030
:1084A000A41500200200000408B50848016B012251
:1084B00011430163006B01211040009000220A204B
:1084C000FEF71CFD0A20FEF70DFD08BD001002405E
:1084D000F0B587B014216846FCF769FE4748C26AC8
:1084E00004210A43C262C26A0A400592C16A802618
:1084F0003143C162C16A31400591C16A01242143FF
:10850000C162C16A21400591C16A02252943C16245
:10851000C06A22462840059005201C210007FEF76E
:108520005EFA012236493748FEF759FA00223649E9
:108530003448FEF754FA9121052000220902000771
:10854000FEF74DFA31480190002705206946029751
:1085500000940007FEF77AF90C200090112001909A
:10856000032003900520029769460007FEF76EF985
:1085700010206A46039591C2052069460007FEF760
:1085800065F91120019002976946039700941D48F0
:10859000FEF75CF91E48019069460095029419485F
:1085A000FEF754F9E00200906946019702951548DC
:1085B000FEF74CF91748694691C16946114803977F
:1085C000FEF744F991200002694691C105206946F1
:1085D00000070397FEF73AF969460A4801970096A3
:1085E0000294FEF733F9002201210520FEF786FCF4
:1085F0000520FEF777FC07B0F0BD00000010024038
:1086000001020000000400500830000000001110BA
:10861000000021100832000010B50F4C0D482060FA
:10862000FF20053060600020A060E0602061606194
:10863000E0610121206249026062A161A06207201D
:10864000E0622046FFF7A7F8206801684022114346
:10865000016010BD003001403016002000B585B02B
:1086600014216846FCF7A3FD0E480D490160E12185
:108670004902416000218160C160016181610C2279
:10868000C1614261016230214162012109038163BC
:108690004900C163FFF794FA00F0F2FC05B000BD99
:1086A00000380140C816002070477047F8B53249BD
:1086B0003048086001F094FD304800F099F8304CE3
:1086C000E0822E48801C00F093F820832B48001D88
:1086D00000F08EF860838B212A4889004180014692
:1086E00040310979284F0906090E617006D1C7800B
:1086F0000121C1870A214187002181872349432223
:108700000A70C18F2171818F6171817AA170858812
:10871000052165626181C6883046FCF7E9FCA081CD
:1087200001462846FCF7E4FC8800081885B2164884
:1087300025816843FCF7B8FF154A164BFCF700FF8C
:10874000FCF7D4FFE081658231463846FCF7D0FC67
:1087500020820146C820FCF7CBFCE0830120A083E7
:10876000FDF79CFBA082E2890B490C48FEF758FB01
:10877000F8BD0000AD90000868000020004F000820
:108780003C010020E40D0020E80300001800002058
:10879000F853E3A59B843E40FF7F000000160020B5
:1087A00070B586B014216846FCF701FD01250F4E17
:1087B000ED03002229463046FEF711F9012000247E
:1087C000019002946946009503943046FEF73EF806
:1087D0000320019002946946009503943046FEF709
:1087E00035F8022000F0CBFE06B070BD000400504A
:1087F0000088704770470000F8B5044600206A46BC
:108800001080194D55222A70AA226A700322AA707C
:10881000661DEE702A716971144A49008918AC719D
:108820002246E81DFCF7AAFC002007E029186A464A
:108830008978128889186A461180401CB042F5DB9D
:10884000611DA81CFDF79EF90146684601802919A3
:108850000078C8716846407808722146093102489C
:1088600000F03AFAF8BD00003E150020E40D0020AB
:10887000034A1168382389B2994301431160704754
:108880000030014010B5FEF7B7F810BD10B59AB032
:1088900034216846FCF78BFC14210DA8FCF787FCFB
:1088A0001C2112A8FCF783FC1B4801680324E40286
:1088B000A143C21489180160FEF72CFB1748016917
:1088C000A143016106200090FF20013002900120A9
:1088D0000390102004900220099040040B900001A6
:1088E00000240C900A946846FEF742FD0F200D907C
:1088F00003200E900F941094012111940DA8FEF7FF
:108900000DFC81201290032080041890149412A86A
:10891000FEF752FB1AB010BD00700040401002403C
:1089200010480168821511430160C1680E4A114068
:10893000C16001680D4A1140016081684908490021
:10894000816001680122920491430160C168FD22A7
:1089500012049143C1600021016106490448886006
:1089600070470000001002400C40FF88F6FFF6FE42
:108970000050000800ED00E010B5CB06DB0E012131
:10898000046A99408C430462016A9A40114301626F
:1089900010BD10B5818CC90707D001684A68012352
:1089A0005B049A43836A1A434A60818C890707D51E
:1089B00001684A6801231B049A43C36A1A434A6048
:1089C000818C490707D501684A6801239B049A43B3
:1089D000036B1A434A60818C090707D501684A680E
:1089E0000123DB039A43436B1A434A60818CC90617
:1089F00007D50268916801231B039943836B1943D0
:108A00009160818C890607D501688A6801235B0320
:108A10009A43C36B1A438A60818C490612D5036856
:108A20005A6801210905046C8A4322435A60026C8A
:108A30008A4207D10268516803235B059943436C5E
:108A400019435160818C090607D501684A680123E2
:108A5000DB04806C9A4302434A6010BDF8B50446BB
:108A6000002680300660FDF7C1FF054620680068DB
:108A7000124F000709D501212B4600224905204647
:108A8000009700F0A1FA00280DD120680068400787
:108A90000BD501212B46002289052046009700F0C6
:108AA00093FA002801D00320F8BD2020A067E067DA
:108AB0002666603426750020F8BD0000FFFFFF0128
:108AC000F8B5154CC826E078002823D16079002835
:108AD00020D101206071114D686B0027002818D04B
:108AE000686BC821081A0FE00D48E168405C6169B5
:108AF0008847E068401CE060E068C82800DBE76069
:108B0000696BC820401A761EE168814201D0002EB0
:108B1000EADC6771F8BD000054000020000002404C
:108B20001C0D002070B5224CE07800283FD1207940
:108B300000283CD1012020711E4EF1690025090654
:108B4000002933DA2156625791420AD1F069400672
:108B50002CD5A079002829D0A5712089401C20811E
:108B600024E0A179002903D1A0710A2000F00EFDB4
:108B700000202056CC2148430F4942182069121882
:108B80001279B262401C00222061A256CC235A43C3
:108B9000895881420ADC25612078401C20702078A9
:108BA0000E2800D12570A078401CA070257170BDE2
:108BB0005400002000380140F401002010B5806A04
:108BC0000022014640314A834A82FEF7E7FE10BD8B
:108BD00070B5846AA06FE56F216889680026090670
:108BE000002906DA212804D152200653204600F03D
:108BF0006BF820688068400606D5222D04D15A20E3
:108C00000653204600F047F82046803001681022C5
:108C1000114301602046FEF7C1FE70BD10B501464C
:108C20000968806A096889061CD400225A210A5200
:108C300001680A68FF2301339A430A6001688A6861
:108C4000520852008A6001688A6840239A438A6009
:108C50002021C167016E012904D101680A6810232F
:108C60009A430A60016E012902D0FFF779F810BD1E
:108C70005821095AFEF790FE10BD10B5806A016EAA
:108C8000012902D0FFF76DF810BD5821095A490893
:108C9000FEF782FE10BD01680A68FF2321339A4364
:108CA0000A6001688A68520852008A60016E0129D0
:108CB00004D101680A6810239A430A602021C16721
:108CC000002101664166704701680A68C0239A4323
:108CD0000A6020218167704770B5164CE278002A3F
:108CE0000CD12279002A09D10122E2700025C8297D
:108CF00003DC0222A256002A01DCE57070BD0123CC
:108D0000E356CC2253430C4AD1500123E356CC26E0
:108D100073439B180A460146181DFCF72FFA60782A
:108D2000401C607060780E2800D16570A078401EED
:108D3000A070E2E754000020F4010020F8B50446DA
:108D4000016880682369E669184363690025334335
:108D50001843724A0B68724E334003430B6021681C
:108D6000486803231B039843E3681843486021685D
:108D7000A069914201D0236A18438B680B26360202
:108D8000B34303438B606749236867488B420CD128
:108D9000C0688007800F06D0012839D0022835D05E
:108DA000032821D11EE001271FE060498B420AD130
:108DB000C0680C21084027D0042829D0082825D0D5
:108DC0000C2811D10EE093420ED1C168032080021D
:108DD000014019D001208002091A19D0091A15D0B2
:108DE000814201D1082700E010274F4950484039FF
:108DF0008600934232D1002F0CD0022F0DD0042FC9
:108E000010D0082F7FD126E00027EEE70227ECE7FD
:108E10000427EAE7FEF750FA06E00968C90605D418
:108E2000304603E0FEF768FA002872D0626851000D
:108E30005118814267D81103814264D3010E0602A2
:108E40005008002330185941FCF768F90321090242
:108E5000411A384A55E00120C003E7E70122E369DF
:108E6000D20393422BD13B0000F0E1F90906090C33
:108E70004D114D4D4D274D00FEF71EFA09E0FEF74E
:108E80002BFA06E00968C90605D4304603E0FEF770
:108E900033FA00283DD0616840004A088018FCF78A
:108EA00027F980B20146244A103991422BD8511C2F
:108EB00001400007400F084329E01046EBE73B0064
:108EC00000F0B5F90906090C211221212123210006
:108ED000FEF7F2F90AE0FEF7FFF907E00968C906B4
:108EE00006D4304604E00EE0FEF706FA002810D063
:108EF00061684A081018FCF7FBF880B201460E4A78
:108F00001039914203D9012503E01046F0E72168AA
:108F1000C86000206066A0662846F8BD0048004092
:108F2000F369FFEF00380140401002400044004068
:108F300000093D00FFFC0F00EFFF0000F8B50446FC
:108F40004165403000262746028380373E6022205C
:108F5000E0672546206F603500281CD01749C162A4
:108F6000216F17480863216F16484863206F866396
:108F7000236F606D9C46134621680246604624318B
:108F8000FDF78CFB002806D0102038602E752020BD
:108F9000A0670120F8BD2E7520680168FF2201320C
:108FA00011430160206881680122114381602068BB
:108FB00081684022114381600020F8BD1D8C0008AB
:108FC0007B8C0008D18B0008FFB581B005460F46A9
:108FD000044660350A9E39E0701C37D0FDF706FD67
:108FE0000499401AB04222D8002E20D0206801688F
:108FF00049072BD5C069C043000527D4012021684B
:10900000C002086220680168FF22A132914301601A
:10901000206881684908490081602020A067E067D6
:109020008034206000202875032005B0F0BD206842
:109030000168FF22A13291430160206881684908DC
:10904000490081602020A067E067EBE72068C169E4
:109050003846884305D0002103988142BCD00020C7
:10906000E3E70121F8E7000010B504491020096882
:1090700008620248FEF794FC10BD0000C8160020EC
:1090800001490D20887070475400002010B5FFF78B
:109090000BFAFFF7E3FAC82202490348FEF730FE55
:1090A00010BD00001C0D0020C8160020F8B53E4C75
:1090B000002321783D4A1D46082910D0072947D0B2
:1090C000062950D0052952D0042953D0032954D061
:1090D000002956D0012958D002295AD05BE0A17846
:1090E00000264A1F04E0314FBF5DFB189BB2761C7F
:1090F0009642F8DB667927799A195118E3786278F5
:10910000C9188918C9194018C0430006000E1AD1A1
:10911000012E14D0022E16D125482449C018FCF780
:109120002DF801F0B9FD642000F029FABFF34F8F4C
:1091300021492048C860BFF34F8F00BFFDE75908A1
:109140001046FFF759FB2570E570A570A571F8BDB5
:10915000A1795054491CC8B2A071A178491F884216
:10916000F5D1082001E0607007202070F8BDE070A4
:109170000620FAE760710520F7E7A070E57004208B
:10918000F3E7552807D10120EFE7AA2803D10220F1
:10919000EBE7032803D02570E570A570F8BD032028
:1091A00020702071F8BD000034010020DA14002086
:1091B000E40D00200400FA0500ED00E010B5024ABD
:1091C000024900F0CDF910BDD1A0000884010020B3
:1091D0002021020C01D010211046020A01D01046B5
:1091E0000839020901D01046091F820801D0104633
:1091F000891E420801D0881E7047081A7047F8B5CA
:10920000040C8BB2264682B25E430D0C1046370C1E
:109210005843360480190021794116466E43370CB5
:1092200036048019794126466E438919F8BD30B459
:109230007446641E2578641CAB4200D21D46635DF3
:109240005B00E31830BC18474900CA020243100013
:1092500000D004204A0D01D001221043044A490DD8
:10926000914201D102210843012800D10520704715
:10927000FF0700008307FF22DB0E9A408907090ED3
:109280009940002808DB830809489B001B181868D0
:1092900090430843186070470007000F08388308A0
:1092A00004489B001B18D86990430843D861704755
:1092B00000E400E000ED00E0F8B504464F1EC800F1
:1092C0000838211815461E46086849683A4606239C
:1092D0009A4310D02A463346FCF7CAF83A46D200E1
:1092E000083AA3181A687F1E5B68FCF70FF806227D
:1092F0003B469343EED1022F23D0042F11D0062FEB
:109300002FD12A463346FCF7B3F8E36AA26AFBF78B
:10931000FDFF2A463346FCF7ABF8636A226AFBF787
:10932000F5FF2A463346FCF7A3F8E369A269FBF789
:10933000EDFF2A463346FCF79BF863692269FBF789
:10934000E5FF2A463346FCF793F8E368A268FBF78B
:10935000DDFF2A463346FCF78BF863682268FBF78B
:10936000D5FFF8BD002210B5134610460149FCF7A1
:10937000E7F810BD0000F03F10B5FBF7C7FF10BDC8
:10938000002210B5134610461146FCF7D9F810BD5F
:1093900010B50721024A00200907FCF749F910BD62
:1093A00001030000034A10B500201107FCF740F943
:1093B00010BD000001FDFFFF02E008C8121F08C138
:1093C000002AFAD170477047002001E001C1121F46
:1093D000002AFBD170470000014908607047000077
:1093E0008801002038B504466D20694608706B4638
:1093F000012207492E2000F029FE0649002C01D049
:10940000054A00E0054A2E2000F006FE38BD0000A7
:1094100006080000061800000706000007160000F6
:1094200010B5002000F006F800220421362000F0DC
:10943000F3FD10BD38B504466B46022200213620EC
:1094400000F072FDB3212300FFF7F1FE0E0F0815A7
:109450003A3A3A3A1C273A3A2F34483A00216846B9
:10946000017040784108490014E069460878800896
:109470008000401C04E06946087880088000801C59
:1094800008701DE0684602780A4048320270417850
:10949000802001436846417012E0684602780A4025
:1094A000027040784106490EF4E769464878022187
:1094B000084303E069464878FD2108406946487042
:1094C0006B4601220021362000F0C0FD012200ABD6
:1094D00011463620013300F0B9FD38BD69460878E1
:1094E000CF21084069462030CAE708B50321684605
:1094F0004170012101706B4602220021362000F0EC
:10950000A5FD0122D20306212D2000F085FD0120BA
:1095100000F035F80120FFF78DFF08BD08B5020AFD
:1095200069464A7008706B46022204212D2000F023
:109530008DFD0320694608706B46012206212D200F
:1095400000F084FD0020694608706B460122062168
:109550002D2000F07BFD0A212D2000F0CBFC08BD62
:10956000F8B516460F460446002503E03946B047D5
:10957000641C6D1C20780028F8D12846F8BD7D2198
:1095800010B5C900484300F001F810BD002140E0CB
:1095900000BF00BF00BF00BF00BF00BF00BF00BFD3
:1095A00000BF00BF00BF00BF00BF00BF00BF00BFC3
:1095B00000BF00BF00BF00BF00BF00BF00BF00BFB3
:1095C00000BF00BF00BF00BF00BF00BF00BF00BFA3
:1095D00000BF00BF00BF00BF00BF00BF00BF00BF93
:1095E00000BF00BF00BF00BF00BF00BF00BF00BF83
:1095F00000BF00BF00BF00BF00BF00BF00BF00BF73
:1096000000BF00BF00BF00BF00BF00BF00BF00BF62
:10961000491C8142BCD37047FFB581B01E460F463E
:10962000040026D00B9903980143A06A394382684D
:1096300007209047002818DB0A99A06A3143826806
:1096400006209047002810DB25462035A979032FF6
:1096500001D908200143032E01D904200143A06A47
:10966000826809209047002806DA0120C04305B02F
:10967000F0BD0020C043FAE7384600F0FFF8206054
:10968000304600F0FBF860600A9868700398A87094
:10969000EF702E710B9868710020E8E7F7B504466B
:1096A000002090B000900190002C05D06A46062161
:1096B00001F02CFB062803DA0020C04313B0F0BDF4
:1096C0006846407801026846007800040918684638
:1096D00080780818FBF7E8FF054668460391007993
:1096E00001026846C07800040918684640790818E5
:1096F000FBF7DAFF032206460F4692075C4BFCF7A6
:109700003BF807D200225B4B30463946FBF7A2FEFE
:1097100006460F4603229207554B28460399FCF74D
:109720002BF807D20022534B28460399FBF792FEF1
:10973000054603912068FBF7B7FF02460B4630460B
:109740003946FBF7FDFE07460A200791205EFBF72E
:1097500097FF3A46079BFBF78BFE064608200991C8
:10976000205EFBF77BFF0021C943FBF7C2FDFBF73F
:10977000DBFF3246099BFBF7C9FD06910890606844
:10978000FBF792FF02460B4628460399FBF7D8FEEB
:1097900005461A200E46205EFBF772FF2A46334626
:1097A000FBF766FE0C9009911620205EFBF768FF20
:1097B000099B0C9AFBF7AAFD05910A902A463346AD
:1097C00038460799FBF754FE059B0A9AFBF750FEB3
:1097D00005910A901420205EFBF752FF3A46079B42
:1097E000FBF746FE07461C200791205EFBF748FF6B
:1097F0002A463346FBF73CFE0E900B911820205E64
:10980000FBF73EFF0B9B0E9AFBF780FD2A46334683
:10981000FBF72EFE0B910E902069FBF731FF0B9B9F
:109820000E9AFBF773FD2A463346FBF721FE0546E9
:109830000E46E068FBF724FF2A463346FBF766FD39
:109840003A46079BFBF762FD059B0A9AFBF75EFD14
:1098500001229207084BFBF70BFE02460B46129CB7
:109860000898069903C411980CC0002026E7000050
:10987000FFFF5F4100007041E17A843F00B50121A4
:10988000C9040300FFF7D3FC081A05080B0E1114D6
:10989000171A0320C00400BD0720C00400BD0F201C
:1098A000C00400BD1F20400300BD3F20400300BD99
:1098B0007F20400300BDFF20400300BD084600BDDF
:1098C000FEB5264F0D4604000FD0002D0DD02646C4
:1098D00000202036B071F07129680D2088470028DB
:1098E00001DA7800FEBD102801D03846FEBDA56221
:1098F000E968002901D028208847204600F030F888
:109900000028F3DBA06AA52182680E209047A06A98
:10991000962182680F209047A06A02218268622007
:109920009047A06A002182680E209047A06A00211B
:1099300082680F20904771793020019100900623B2
:10994000202201212046FFF767FE0028CEDB2046BB
:1099500000F0AEF80028C9DB0020FEBDFFFFFFFFCE
:1099600010B586B0044614216846FBF720FC002C95
:109970007ED0A06A122143686A46102098471228B8
:1099800077D16846007801220101684640781203C9
:109990000009081843492081884201DD801A20818E
:1099A0006846837840780007000D18186081884267
:1099B00001DD801A60816846007901220101684654
:1099C000C078120500030918684640790009081894
:1099D0003549E060884201DD801AE06068464079E0
:1099E0000007030B6846807900021B186846C0799F
:1099F00018182061884201DD801A20616846417A8A
:109A0000007A0002081802B2284801210904A28243
:109A1000824201DD521AA2826A46D37A927A1202F7
:109A20009A1812B2E282824201DD521AE2826A463A
:109A3000537B127B12029A1812B22283824201DDFA
:109A4000521A22836A46D37B927B12029A1812B270
:109A50006283824201DD521A62836A46537C127C21
:109A600012029A1812B2A283824204DD501A01E057
:109A70000BE008E0A083A06A01682820884700283E
:109A800006DA0120C04306B010BD0020C043FAE74B
:109A9000C011C0072034002800D080206071002051
:109AA000F1E70000FF070000FFFF0700FF7F000055
:109AB00010B5040009D0A06A0721826808209047E9
:109AC000002805DA0120C04310BD0020C04310BDAE
:109AD000072020342070002010BD000038B5044657
:109AE000FFF79EFCFF2252030021282000F09FFA7E
:109AF0000E4A0021282000F09AFA0220FFF79AFC73
:109B00000D20FFF797FC042C00D2042422460021EC
:109B10000A2000F08CFA1020694608706B4601227A
:109B200024212F2000F092FA38BD000000FF5F00D2
:109B3000FEB5044600200190009060797349400012
:109B40000E5A61782578491E7148CFB20163042D01
:109B500077D0072D75D000210291217801736C49CF
:109B6000E379012292058969002B6CD091438161D0
:109B70006748217A4173217A82698907890B0A43F0
:109B800082610021042000F052FA324661492E2001
:109B900000F042FA3846FFF725FC5F4E0522705D63
:109BA000810040185D49431807212B2000F04EFA30
:109BB0005B49029801220B180B21282000F046FA7D
:109BC000705D584980000A580C21282000F02FFAB7
:109BD000E079554980004018A1794900425A022194
:109BE000272000F019FA51487E00825B04212720CB
:109BF00000F012FAE079002829D0A07804282CD0AF
:109C000028206946087220220621272000F004FA45
:109C100002AB01222621272000F018FA444938011E
:109C20004018E178890042580821272000F0FFF908
:109C3000A17A601C627A0902114313D016E000E099
:109C400001E0012188E71143F608816190E7642271
:109C50000621272000F0E0F9E0E7102069460872AD
:109C60000246D1E733490172090A4172417A007A0A
:109C70000A0202432021272000F0CEF92E4F0C21AA
:109C800023203A6800F0D3F9F019828804212320B8
:109C900000F0C2F9A07900280BD0E0792749012211
:109CA00043180021212000F0D1F903200190012068
:109CB00000902A07120F10010243607800218007EC
:109CC000000B024301980005024300984004024340
:109CD0002079C006400902436079C00602431F2074
:109CE00000F0A5F9A0786178012308430204084830
:109CF000DB030261E179490319430A430261002150
:109D0000082000F094F90020FEBD000040AE0008DD
:109D1000B801002004280000E8AD0008240000205D
:109D200042000020F0AD000810AE00081CAE000894
:109D300020AE00084110000008AE000844000020DA
:109D400010B504460421362000F0D4F80121C902E0
:109D5000002C01D0084300E088430246042136204D
:109D600000F065F910BD0000FEB505460420694607
:109D70000870514C002060752146203120634871E5
:109D80000873A0836063A06300F0C8F84B4E2060A6
:109D900002E000F0C3F82060B042FAD10020FFF7E3
:109DA00049FB00F0BBF8464E20603078242801D9EA
:109DB000243806E00621FBF79BF90622101A400121
:109DC0000843020601040A4301020A430243B26047
:109DD000706000211E2000F02AF900F09FF820603A
:109DE0006B4601220021242000F030F91E20FFF7ED
:109DF00095FB86B2300AA0730420FFF78FFB07465D
:109E000000F08CF820603806000E0DD00220694664
:109E1000087101AB012212212D2000F017F9A08B4F
:109E2000012109030843A08300F078F82060062090
:109E3000FFF774FB60600720FFF770FBA060F0067F
:109E4000C00E207501D110202075C0B200F028F995
:109E5000E80707D0FFF749FBA08B0121C90208439F
:109E6000A0830AE00521362000F02EF815490840AD
:109E700002460521362000F0CFF80120FFF7DAFA7C
:109E80000021042000F036F8A0610021262000F017
:109E900031F815218903084302460021262000F0ED
:109EA000C6F800222621362000F0B6F800F036F879
:109EB00020600020FEBD0000B80100203001CADE95
:109EC00018000020FFFD000038B5094C89B280B2AF
:109ED0006B46022200F028F8002806D16846407838
:109EE000010268460078081884B2204638BD000098
:109EF000FFFF000038B50024E44389B280B26B460E
:109F0000042200F011F8002806D103216846435CC2
:109F10002202D418491EFAD5204638BD10B50021BA
:109F20000846FFF7E7FF10BD38B5002909D04024E7
:109F300020436C462070C8B27F2906D8607002208A
:109F40000AE069460870012006E0802420436C4640
:109F50006070C809A0700320694600F077FE38BD24
:109F600010B5024602492E2000F056F810BD000040
:109F70000418000010B502460021182000F04CF82B
:109F800010BD0000F8B50746002568460570B80703
:109F9000204C2E4600280ADA8020694608706B465D
:109FA000012200210D2000F051F801202073F80754
:109FB0006946087821D006210843694608706B4637
:109FC000012200210D2000F041F803210F20FFF7AE
:109FD0007BFF8121C900084219D0402069460870E2
:109FE0006B46012200210D2000F030F80020FFF721
:109FF000A7FE00252673ED4309E0022108436946C8
:10A0000008706B46012200210D2000F01FF8284641
:10A01000F8BD0000D801002008B56B461A70120A7E
:10A020005A7089B280B2022200F010F808BD38B52B
:10A0300000236C46E254120A5B1C042BFADB89B243
:10A0400080B22346042200F001F838BD38B58024E0
:10A05000002909D0C02528436D462870C8B27F2941
:10A0600007D86870022009E0204369460870012083
:10A0700004E020436870C809A8700320694600F016
:10A080008FFE38BD10B5054A8905126901430A43A0
:10A0900000210820FFF7CBFF002010BDB8010020F1
:10A0A00038B504466B4601220E212B20FFF73CFFFA
:10A0B00068460078E10640094001C90E0143684640
:10A0C00001706B4601220E212B20FFF7BFFF38BD28
:10A0D00013B501231A4669460248FDF743FE00986E
:10A0E0001CBD0000C8160020FCF78EFCFEF7CEFB5E
:10A0F000FEF7EEF9194818490160002141608160BE
:10A100000162174A416242618162FCF70FFEFEF76D
:10A11000CBF9FEF7A3FAFEF77FFAFEF791F90122D9
:10A120000520D1030007FCF75AFCFEF7BFFAFEF743
:10A130006FF8FBF703FDFBF785FDFBF753FD0948BF
:10A14000FFF7CCFC00210D20FFF79CFF0020FFF75C
:10A1500019FFFDF783FFFCE7007C0040001600209C
:10A16000FFFF000080E7010010B586B01748FCF73C
:10A1700060FD14216846FBF71AF81548009003208B
:10A18000019000200290052069460007FCF75EFB65
:10A1900069461048FCF75AFB69460F48FCF756FB26
:10A1A00001210846FCF7D6FEFF2401342046FCF7C7
:10A1B000A9FE0A4908680422104308602046FCF7FB
:10A1C000B1FEFCF7B7FE06B010BD0000001600207F
:10A1D000FFFF000000040050000800500070004025
:10A1E00010B50122920217491748FBF7ADFD15483B
:10A1F000164902888A4223D0018004218180FF21F0
:10A20000F531C1800A21018100211E224181D24302
:10A2100082810122C28181834323C3860223038773
:10A22000782343878287C287024640321184518453
:10A230009184C183918014238382118200F02CFDCC
:10A2400010BD0000E40D002000FC0008AA5500002D
:10A25000F0B51FB496B084460C460246199D189876
:10A260000390490068006300490840080193002AF0
:10A2700001D0012600E000269E19FE4BF6185B1067
:10A280009E422BD36E00039F0296002F00D0012721
:10A29000F719F84EF84BBE199E421FD3039E034692
:10A2A000F64F334309D03B469C4201D1002A04D0EB
:10A2B000019B002A05D0012604E0002039461BB08E
:10A2C000F0BD00269E19EE4B9E4207D8039F029ECA
:10A2D000002F00D00127F6199E4207D92B46604671
:10A2E0002146189AFFF748F81BB0F0BD0023002C58
:10A2F00029DAE44EB04226DAE34EB04201DB022313
:10A3000021E0DE4EB0421EDBE04E070DBE19142EDA
:10A3100009DD3427BF1B039EFE400196BE40039F0C
:10A32000BE420BD00FE0039F002F0CD11427BF1BA0
:10A330000646FE400196BE40864204D1019BDE07E0
:10A34000F60F02239B1B0E46164318D1002D16DA7A
:10A35000002C03D0022B01D0012B06D00220FFF7E6
:10A360003BF8FEF7FFFF1BB0F0BD0220FFF734F80B
:10A37000FEF7F8FF0122D20751401BB0F0BD039E4B
:10A38000002E61D1BF4EB04220D1C148844201D1DC
:10A39000002A08D0B948814209DB002D10DB18984B
:10A3A00029461BB0F0BD0020B4491BB0F0BD002D04
:10A3B00006DA01222946D207189851401BB0F0BD99
:10A3C000B4497944086849681BB0F0BDAB4FB84246
:10A3D00025D1002D1FDA002904D0B14212D1002A64
:10A3E00009D018E0002A72D1A649E20F0020D20756
:10A3F00011431BB0F0BD0020E20F0146D20711430C
:10A400001BB0F0BDB14206DA234600203946FBF707
:10A4100097F81BB0F0BD104621461BB0F0BDB1420D
:10A4200012DA0126B607B54203D123461046194673
:10A43000FEE3994EB54207D1261E05DB1046314694
:10A4400000F040FC1BB0F0BD67007F081646002AF4
:10A4500040D100290AD08B4A914229D1002C0EDD2F
:10A46000002D1CDB002011461BB0F0BD022B16D0C6
:10A47000002C14D0012B12D1002C14DB0FE0002C87
:10A4800028DA002D09DB012B03D000207D491BB009
:10A49000F0BD002081491BB0F0BD012B03D000208E
:10A4A00001461BB0F0BD00200121C9071BB0F0BD63
:10A4B000724A91420ED1002C01DA002B17D0022BE8
:10A4C00006D00020C043FBF7DBF81BB0F0BD90E2E4
:10A4D0000120F8E7E217521C94461A4307D00022E5
:10A4E0000892664C62465B1E1A4307D009E00120C1
:10A4F000FEF772FFFEF744FF1BB0F0BD0022644C74
:10A500000892674A90427DDD664B674A98421FDD9C
:10A51000914202DC002D05DB4DE05848814217DBFB
:10A52000002D48DD0220FEF757FFFEF731FF0546FC
:10A530000E460022534B21460898FAF799FF084629
:10A5400071004908C00FC007014328461BB0F0BD89
:10A55000914215DA002D2EDA0220FEF73DFFFEF7BC
:10A5600017FF05460E460022464B21460898FAF78B
:10A570007FFF72005208C80FC0070243114617E060
:10A580003E4B994223DD002D15DD0220FEF724FF0E
:10A59000FEF7FEFE05460E4600223A4B214608987D
:10A5A000FAF766FF084671004908C00FC00701436B
:10A5B00028461BB0F0BD0220FEF70EFFFEF7F2FEAC
:10A5C00049004908E20FD20711431BB0F0BD002239
:10A5D00030463946FAF73EFF012205460E46D24381
:10A5E000FBF726F8314A324BFAF73AFF2A46334650
:10A5F000FAF73EFF0022284BFAF732FF07462A46B9
:10A60000334600E064E0039110461946FAF730FF44
:10A610003A46039BFAF72CFF07460322099152079B
:10A62000244B28463146FAF723FF07910C90224A23
:10A63000204B38460999FAF71BFF074601911F4A3C
:10A640001F4B28463146FAF713FF3A46019BFAF7AB
:10A6500001FF07460B460246099107990C98FAF745
:10A6600055FE00250E462846079B0C9AFAF7F2FE87
:10A670003A4627E0FFFF1F00FFFF0F000000F03FFA
:10A680000000E0FF0000F07F0000404301FCFFFFFE
:10A690000000F0BF5A0B00000000E03F0000F0FF98
:10A6A0000000E0410000F043FFFFEF3F55555555D6
:10A6B0005555D53F4715F73FFE822B6544DF5DF8C2
:10A6C0000BAE543E099BFAF7CBFE02460B4652E115
:10A6D000012500202D05A94207DA352230463946EA
:10A6E000FAF7A6FF06463420C0430A151218FE48A2
:10A6F000101803900803FD49000B01430F46FC4965
:10A70000884201DC002003E0FA49884202DA012095
:10A71000119005E0002011900398401C7F1B0390CE
:10A7200011980597C200F4480F9278448018436846
:10A730000268394630460D930292FAF78BFE079174
:10A740000C9030460D9B029A0599FAF7DFFD024600
:10A750000B460020E549FAF7F3FE09910490079BA8
:10A760000C9AFAF785FE129000201090E3480D46EF
:10A77000784400680E900121781049070843119928
:10A780000D9B890440180121C90447183946029AD3
:10A790000E98FAF75FFE3246059BFAF761FE024615
:10A7A0000B4629461098FAF763FE064602913B468F
:10A7B00029460E9A1098FAF75BFE079B0C9AFAF757
:10A7C0004FFE3246029BFAF745FE099B049AFAF7C0
:10A7D0004FFE0591129A0A902B4610461946FAF739
:10A7E00047FE06460246C6480F460B4606217844F9
:10A7F000FEF762FD32463B46009104901046194632
:10A80000FAF736FE009B049AFAF732FE06460F4628
:10A810002B461946129A1098FAF778FD059B0A9A6A
:10A82000FAF726FE32463B46FAF770FD109A07917A
:10A8300004902B4610461946FAF71AFEB14E002234
:10A84000334609910290FAF761FD079B049AFAF7E3
:10A850005DFD00200746024633460091FAF7FAFDF7
:10A86000099B029AFAF7F6FD079B049AFAF7F8FD9E
:10A8700006460D913A462946009B1098FAF7F8FDD6
:10A8800007910C902B463046129A0D99FAF7F0FD7D
:10A8900005460E463A46009B05990A98FAF7E8FDE8
:10A8A00033462A46FAF732FD02460B46074609911F
:10A8B00007990C98FAF72AFD00250E462846079BB3
:10A8C0000C9AFAF7C7FD3A46099BFAF7C9FD074605
:10A8D0000722099152078C4B31462846FAF7C8FDEA
:10A8E00007910090894A884B38460999FAF7C0FDCC
:10A8F00007460191864A874B31462846FAF7B8FD4C
:10A900003A46019BFAF702FD834B7B440F9A9B1852
:10A910001A685B68FAF7FAFC029009910398FAF753
:10A92000AFFE05910490099B029A07990098FAF7E7
:10A93000EDFC7A4B7B440F9A9B181A685B681746AC
:10A940000393FAF7E3FC059B049AFAF7DFFC0E4643
:10A950002846059B049AFAF77DFD3A46039BFAF7D1
:10A9600079FD079B009AFAF775FD099B029AFAF7A1
:10A9700077FD02460B46199900200C900F46189857
:10A98000FAF776FD029104903B460C9A19991898B3
:10A99000FAF760FD2A463346FAF76AFD029B049AED
:10A9A000FAF7B4FC09910E902A46334639460C98C2
:10A9B000FAF75EFD06460F46099B0E9AFAF7A6FCCB
:10A9C000574A0D46914220DB5242AA18024310D149
:10A9D00032463B46FAF73EFD04900391514A524BF2
:10A9E00009990E98FAF792FC039B049AFAF7C4FEB1
:10A9F0001ED20220FEF7F0FCFEF7CAFC490049080F
:10AA0000E20FD20711431BB0F0BD6A00474B52085A
:10AA10009A420DD3464AAA18024300D0CBE53246EB
:10AA20003B46FAF717FD099B0E9AFAF7A5FEF5D9F2
:10AA30006800002340082C490393020D3D4B521837
:10AA4000984223DD01200005521CD04042195000DD
:10AA5000400D401838497944096813468C463749F7
:10AA6000C1408B4312030121120B09055118142216
:10AA7000101AC1400391002D01DA4842039062464A
:10AA800030463946FAF7E6FC06460F4632463B4664
:10AA900009990E98FAF73AFC00252A46284B2846D1
:10AAA0000591FAF7E5FC07910C90264A264B2846BB
:10AAB0000599FAF7DDFC0091029032463B462846A4
:10AAC0000599FAF7C7FC099B0E9AFAF7C9FC1F4AC9
:10AAD0001F4BFAF7CDFC009B029AFAF717FC0746CA
:10AAE0000B460246099135E001FCFFFF0000F03FF4
:10AAF0008E9803007AB60B006A070000AC070000CE
:10AB0000D60600000000084009C7EE3FFD033ADC0E
:10AB1000F5015B14E02F3EBEAA05000070050000A1
:10AB200000009040FE822B654715973C00CC90407A
:10AB300000346F3F0000E03FC6040000FFFF0F003D
:10AB4000432EE63F396CA80C615C20BEEF39FAFE5B
:10AB5000422EE63F07990C98FAF7D8FB05460E46B9
:10AB6000079B0C9AFAF776FC3A46099BFAF778FCB1
:10AB700009912A4633460E9010461946FAF778FC9A
:10AB8000074602462F480B46059105217844FEF7FB
:10AB900093FB3A46059BFAF76BFC2A463346FAF7D5
:10ABA0005FFC0746019128463146099B0E9AFAF749
:10ABB0005FFC099B0E9AFAF7A9FB012304910C9004
:10ABC00000229B0738460199FAF744FC05910E9044
:10ABD0003A4628463146019BFAF74AFC059B0E9AF5
:10ABE000FAF7AEFC049B0C9AFAF734FC2A4633467B
:10ABF000FAF730FC0022144BFAF732FC06460398B1
:10AC00000D46000541190915002912DC3046294678
:10AC1000039AFAF70DFDFEF717FB042801D1FEF7A2
:10AC2000C1FB30462946039AFAF702FD064601E0C9
:10AC300004E029180B46324621460898FAF718FC1A
:10AC40001BB0F0BD680300000000F03FF0B58C467B
:10AC500000251026052109078E620E4C08E0674684
:10AC60007F5DE760A768FF07FCD0E7681F706D1C79
:10AC70008542F4DB0020074606E0E760A568ED07A3
:10AC8000FCD0E5681D54401C9042F6D38E61002034
:10AC9000F0BD00000030014070B572B60124074DD0
:10ACA000A40221462846FBF735F8002804D02246A6
:10ACB00003492846FBF7D2F862B670BD00FC0008D5
:10ACC000E40D0020F8B506460C46FAF763FE051EB3
:10ACD0000F4600D00120014349000B484908411AA2
:10ACE000C90F0DD0002E01D0012100E000210C433E
:10ACF00061004908401AC00F02D10120FEF76CFB29
:10AD000028463946F8BD00000000F07FF8B515462A
:10AD10000E460746002407E03819C0B200F008F8D4
:10AD2000641C2870E4B26D1CB442F5D33046F8BD03
:10AD300010B50446FDF72EF9EE20FDF7FEF8FDF7FD
:10AD400062F92046FDF7F9F8FDF75DF9FDF722F904
:10AD5000EF20FDF7F2F8FDF756F90020FDF7C0F8F7
:10AD60000446FDF732F9204610BD704770B50D4618
:10AD70000446FDF70FF9EE20FDF7DFF8FDF743F984
:10AD80002046FDF7DAF8FDF73EF92846FDF7D5F83D
:10AD9000FDF739F9FDF719F90A20FEF7F7FB70BD49
:10ADA000F0B50025102605279C463F070B46BE62DE
:10ADB0000C4C06E0595DE160A168C907FCD0E16870
:10ADC0006D1C8542F6DB002007E06146095CE1600E
:10ADD000A168C907FCD0E168401C9042F5D3BE6170
:10ADE0000020F0BD00300140000001020304000516
:10ADF000405C0000A05C0400C06C0800805C0400A3
:10AE0000E03F1E00E07D1E0007A9022570889B8898
:10AE10000A001600010006000100020087008D00F4
:10AE20002D001A3152001A339A001A351D011A37B3
:10AE30006B003B31BE003B335E013B3596023B3736
:10AE4000000099599959EB518F421E45142E0080EC
:10AE5000EB51F5283333E13A703DE13AC235852BA9
:10AE6000C2353333C235C235AE47E13A5138A3302B
:10AE70005138000000000000000001020304060732
:10AE80000809030406080C10182030000000000117
:10AE90000203040000000000000000000000F03F7A
:10AEA000000000000000F83F00000000000000006B
:10AEB0000000004003B8E23F000000000000000076
:10AEC00006D0CF43EBFD4C3E033333333333E33F04
:10AED000FFAB6FDBB66DDB3F4D268F515555D53F30
:10AEE00001411DA96074D13F65DBC9934A86CD3FFE
:10AEF000EF4E454A287ECA3F3E5555555555C53FEC
:10AF000093BDBE166CC166BF2CDE25AF6A56113FDD
:10AF1000F16BD2C541BDBBBED0A4BE726937663EDF
:10AF2000000000000000000048AF00080000002002
:10AF30008C0100005C5A0008ACAF00088C010020B6
:10AF40006C1A0000C89300080124130704380D0987
:10AF50001E080540082609104008560A131D043B28
:10AF600008BE0516D8BC4010085201033AC8420773
:10AF70007052030CE5800C1B0202DD140901022251
:10AF800081F01F66810498899686967982159803C8
:10AF900098149887967497788243978896719777D4
:0CAFA0008249F10135293B920492200007
:04000005080050C1DE
:00000001FF
